:020000040000FA
:040000000B303A285F
:08000800A000030EA100831209
:100010008B1C32288B1031181428B11C3228643004
:10002000010203183128182800001628172818285C
:1000300019281A281B281C281D281E281F283110A3
:10004000B114A810031005190314AA0DA90DA80DC9
:10005000B00B322831152A08AF002908AE00280855
:10006000AD00B11081010B11210E8300A00E200EF6
:02007000090085
:0C007400203084008001840A6030040207
:10008000031C3C281230B00019228316FF23900075
:1000900083128316851683120C30851A2C30831632
:1000A000850083128501870107309900003083168F
:1000B00091009F008312C830831681008312313073
:1000C0009000003083168C00831210308B00BC1B14
:1000D0006F2885196F286400851D6B28B1223C1C90
:1000E00072287D2281018E018F010B118B100B1064
:1000F0008C018B178A203119A020FD21B30B882891
:10010000031085190314B90DF030390203198F213A
:1001100086227A286400311808000B1D08000B1194
:10012000B11031141230B000051D9B283214831613
:10013000011383120800321083160117831208007E
:1001400031110130B7008B132030370783169B0025
:100150001C141A088312A400A500C030A506103094
:10016000370783169B001C141A088312A300003063
:10017000370783169B001C141A088312A2008B17E2
:10018000321CC82822090339A200A309A409A50921
:1001900022082D02031D892923082E02031D892907
:1001A00024082F02031D2C2901303702031DDF28EC
:1001B0003C19DE283D18DF283D143E14362202305B
:1001C0003702031DEA283C19E928BD18EA28BD14A6
:1001D0003E143D2203303702031DF5283C19F42854
:1001E0003D19F5283D153E14442204303702031D05
:1001F00000293C19FF28BD190029BD153E144B22CA
:1002000005303702031D0B293C190A293D1A0B2919
:100210003D163E14522206303702031D16293C19A2
:100220001529BD1A1629BD163E1453220730370270
:10023000031D21293C1920293D1B21293D173E146E
:10024000542208303702031D2C293C192B29BD1BD1
:100250002C29BD173E14552225082F02031D89297C
:1002600001303702031D3B293C193A293D1C3B292B
:100270003D103E14562202303702031D46293C1918
:100280004529BD1C4629BD103E14582203303702B3
:10029000031D51293C1950293D1D51293D113E1482
:1002A0005A2204303702031D5C293C195B29BD1D0D
:1002B0005C29BD113E145C2205303702031D6729FD
:1002C0003C1966293D1E67293D123E146322063003
:1002D0003702031D72293C197129BD1E7229BD12F6
:1002E0003E14642207303702031D7D293C197C2906
:1002F0003D1F7D293D133E14652208303702031D42
:1003000088293C198729BD1F8829BD133E14662200
:100310008929B70A0530370203180800A3280130DD
:10032000B600B300B400B500B70004308316851AD8
:10033000B700831285018701B1138A20B30BCC2942
:10034000031085190314B90DF03039020319F3298C
:10035000B40BCC290130370203196722023037026F
:1003600003196B220330370203196F22043037025E
:10037000031973220530370203197722063037023A
:10038000031978220730370203197922083037021F
:1003900003197A229630B400311D9D293111321C87
:1003A000D6292D090339AD00AE09AF092F1CB113B1
:1003B0002F1C9D29B11B9D292E189D29B1178B1328
:1003C00020303707BB002F08BA000622103037074D
:1003D000BB002E08BA00062200303707BB002D08EC
:1003E000BA0006228B1785018701B70AB6010530CE
:1003F0003702031C9D297D2208003E1C08003E1088
:100400001030BB003D08BA00062208008B133A08E2
:1004100083161C159A003B089B0055309D00AA309E
:100420009D009C1464009C18122A1C1183128B17C7
:100430000800831600309B001C141A088312BC00AD
:10044000831610309B001C141A0883123C18BD0040
:10045000831620309B001C141A088312C10001303F
:10046000C11BC100C1080319C10008008514400860
:100470004107D0000F08D1000800051440084107CB
:10048000D2000F08D3000800851640084107D400A9
:100490000F08D5000800051640084107D6000F08D0
:1004A000D7000800080008000800080085100800B0
:1004B000051008008512080005128E018F010C102E
:1004C0004108C000080008000800080008000508EE
:1004D000023A850008000508013A85000800050871
:1004E000203A850008000508103A85000800080039
:1004F000080008000800080008003D188514BD1811
:1005000005143D198516BD19051608003C1D080087
:1005100050084002031D912A51080F02031C912A22
:10052000851052084002031D9A2A53080F02031C2B
:100530009A2A051054084002031DA32A55080F02E9
:10054000031CA32A851256084002031DAC2A570833
:100550000F02031CAC2A05120C1C08000C10C00A68
:100560000800B601B301B4013C1CB92ABC01BC149B
:10057000C02ABC1CBE2ABC013C15C02ABC013C14CC
:100580003C08B6006400C42AC52AC62AC72AC82A5D
:10059000B41B8514B41F8510B30BC22AB40BC22A36
:1005A0000310B60CB608031DC22A0030BB003C087D
:0605B000BA00062208005B
:084000000D000300060004009E
:02400E00CC01E3
:10420000010003000300030003000200020002009B
:1042100002000000000000000000FF00FF00FF009F
:10422000000000000000000000000000000000008E
:104230000000C000C000C000C000FF00FF00FF0081
:104240000100C300F300CF00FF00C300F300CF0064
:10425000FF00C300F300CF00FF00FF00FF00FF00DE
:10426000FF00FF00FF00FF00FF00FF00FF00FF0056
:10427000FF00FF00FF00FF00FF00FF00FF00FF0046
:10428000FF00FF00FF00FF00FF00FF00FF00FF0036
:10429000FF00FF00FF00FF00FF00FF00FF00FF0026
:1042A000FF00FF00FF00FF00FF00FF00FF00FF0016
:1042B000FF00FF00FF00FF00FF00FF00FF00FF0006
:1042C000FF00FF00FF00FF00FF00FF00FF00FF00F6
:1042D000FF00FF00FF00FF00FF00FF00FF00FF00E6
:1042E000FF00FF00FF00FF00FF00FF00FF00FF00D6
:1042F000FF00FF00FF00FF00FF00FF00FF00AA001B
:00000001FF
